:020000040000FA
:100000000000000000006C28F100030EF20004085C
:10001000F3000A08F4008A01831203138316031302
:100020000C1E1728831203130C1E17285A20831640
:1000300003138C1E2028831203138C1E20283920C2
:100040000C1C3028DB03031D2A285F170A30DB0055
:100050002030850651308E00C3308F000C103028C0
:1000600074088A0073088400720E8300F10E710E0A
:10007000090018197815781018187814831776085D
:1000800084001A08800000080A3A03195228F60A68
:1000900004086D3A031D0800840A0D308000840AAC
:1000A0000A3080001030F600831603138C1283127E
:1000B00003130800831777088400000883120313D2
:1000C0009900F70A0A3A031D080083160C128312DE
:1000D00003139030F7000800831603138B309F0042
:1000E0003F308500C8308600D830870081018117F5
:1000F000011383120313DD0181309F008B018316EE
:100100000313243098004030990083120313903079
:100110009800F8011030F6009030F7003030900071
:1001200051308E00C3308F000A30DB00831603137A
:100130000C14831203130B1710144830D000061050
:1001400056216821D60100308621562106145621F9
:100150005930862168210B30F5000610562106140F
:10016000562190308621D70109306F218130DD0082
:10017000C3203B218930DD00C3203B21A130DD00BD
:10018000C3206821AD28831203135D089F001F144C
:10019000EA201F15EA20EA20DF131F19CD28831259
:1001A00003131E0883160313B200B6001E08B30023
:1001B000B70083120313DF12DF13BA2109306F2156
:1001C0000800831603133508B3023408031C340FE8
:1001D000B2020800831603130130BC000130BD00D9
:1001E0000A30BE005F29831603130130BC000130C2
:1001F000BD002830BE005F29831603130130BC0008
:100200000130BD005030BE005F298316031301305A
:10021000BC000130BD007830BE005F298316031397
:100220000130BC000130BD00C830BE005F2983161C
:1002300003130130BC000230BD009030BE005F29C6
:10024000831603130130BC000830BD00CD30BE0062
:100250005F29831603130130BC001030BD009A30B3
:10026000BE005F29831603130130BC002830BD0097
:100270000130BE005F29831603130130BC009D309E
:10028000BD000230BE005F29831603130130BC009D
:10029000C430BD000230BE005F2983160313043052
:1002A000BC000E30BD003730BE005F29831603133B
:1002B0000730BC001B30BD007030BE005F29BE0B94
:1002C0005F29BD0B5F29BC0B5F2983120313080054
:1002D000831203130D306F210A306F21080083123F
:1002E000031364000C1E7229990008005F1B7C290F
:1002F0008C1E78291A0808005F132A300800831220
:10030000031364008C1E82291A0808008312031349
:10031000D60056089221D60AFF39031908006F212A
:1003200089290800831203178D00831603178C1385
:100330000C14831203170C08831203130800831292
:1003400003178C00831203135C30831203178D0094
:10035000831603178C130C158B1355308D00AA30A0
:100360008D008C148B1764008C18B3290C11831228
:1003700003130800831603133208B0003308B100DA
:10038000300EF038A500A507E23EA600323EA800D8
:1003900030080F39A607A607A807E93EA700A70758
:1003A000A707310E0F39A707A807A70DA80DA809A1
:1003B000A80D31080F39A807A50D0730A4000A3091
:1003C000A807A703031CE029A707A603031CE42929
:1003D000A607A503031CE829A507A403031CEC2911
:1003E00083120313DF1E192A2030DF1B2D306F21EB
:1003F000831603132508031D032A831203132030D9
:100400006F21DF14072A83120313303E6F218316F6
:1004100003132608303E6F212E306F2183160313FD
:100420002708303E6F21831603132808303E6F21C2
:100430000800831603132508303E6F21831603132B
:100440002608303E6F21831603132708303E6F21A4
:10045000831603132808303E6F2120306F210800D7
:10046000D5008B128B17D8010B165F1F352A5F132F
:100470008B130B1258086F211B305806031D412A9D
:10048000080008305806031D4B2A44305502031853
:10049000322AD50A322A09305806031D542A550338
:1004A0000318542AD503322A303058020318592A27
:1004B000322A39305802031C602A0319602A322A72
:1004C0005518632A742A30305802DA000310DA0D06
:1004D000DA0DDF1A6F2A0310DA0DDA0D722A5A07C5
:1004E000DA00DA0DD503322A303058020F395A07B4
:1004F000D8000310550C443E84005808800055086D
:100500000319852AD503031D322A8B1358080800C6
:10051000892A8A2A8B2A8C2A8D2A8E2A8F2A902A27
:10052000912A922A932A942A952A962A972A982AD7
:10053000992A9A2A9B2A9C2A9D2A9E2A9F2AA02A87
:10054000A12AA22AA32AA42A0800831686138312AA
:10055000861706178822861388220613080083163A
:1005600086138312861306178822861708008316BF
:100570008613831286138822061788220613080022
:10058000831686138312861788220617882206137D
:1005900008008316861783128822061788220315FF
:1005A000861B031106130800EB228822F4228822FE
:1005B000080086178316031300008617831203139F
:1005C0008822080083160313861383120313000086
:1005D00086138822080006178316031300000617E7
:1005E0008312031388220800831603130613831251
:1005F0000313061388220800D2010830D400D92240
:10060000EB22861F042B072B0310D20D0B2B03109C
:10061000D20DD20A0B2BF422D40B002B0800D100F0
:100620000830D4000310D10D031C172B1B2BE22222
:10063000D422D9221E2BD922D4221E2BD40B122B2A
:100640000800AF223221A522D0300F23C922CD01CC
:100650004D080F23C92244080F23C92245080F2340
:10066000C92246080F23C92247080F23C922480878
:100670000F23C92249080F23C9224A080F23C92280
:1006800090300F23C022AF2229210800AF22EA2098
:10069000A522D030CE000F23C922CD014D080F2353
:1006A000C922D130CE00A5224E080F23C022FC2241
:1006B000B7225208C400FC22B7225208C500FC220F
:1006C000B7225208C600FC22B7225208C700FC22FB
:1006D000B7225208C800FC22B7225208C900FC22E7
:0A06E000B7225208CA00AF2208003A
:084000000200010000000000B5
:02400E00323F3F
:1042000031343634463438343734363441345F341C
:10421000523453343234333432342E344134533400
:104220004D34203420343134363420346F34633408
:1042300074342034303439340C340D34503449342F
:104240004334313436344634383437343634203419
:10425000733461346E3473342034203462346F34F8
:104260006F3474346C346F34613464346534723454
:1042700020340C340D347434653473347434203485
:1042800066346F346E346334743469346F346E342E
:104290002034553441345234543420343134393498
:1042A0003234303430346234643473340C340D348A
:1042B0000034333420344D346534733475347234FF
:1042C00065347334203441346E3461342E342034F8
:1042D00020340C340D346134763465346334203446
:1042E0002B345234453446343D3435342E34303456
:1042F00030343D34563464346434203420346534EE
:10430000743420342D345234453446343D34303402
:1043100056343D345634733473340C340D34003415
:104320004C346534633474347534723465347334A6
:0E433000203441344434433473342034003498
:00000001FF
